:10000000012883160F30860000308500831281019D
:100010008B018316C03081008312B301B4015520D7
:10002000060810308B00630006088D2000308B001E
:100030009520061C43280108B500061C25284920E8
:1000400050208D20850186011B2820308620010844
:10005000B50049205020203086200108B5004920F5
:100060005020303086200108B50049205020303023
:1000700086200108B5004920502040308620010824
:10008000B50049205020502080308620850186010F
:10009000102835080739B300350E0739B4000800B9
:1000A00033087E2034088120080085018601013054
:1000B00081208D20023081208D20033081208D20F1
:1000C000043081208D20053081208D200630812054
:1000D0008D2001307E208D2002307E208D20033047
:1000E0007E208D2004307E208D2005307E208D20C6
:1000F00006307E208D208601850108009D20850028
:1001000008009D20B000300E86000800B100B2004B
:10011000B20B8828B10B872808001430B100B20058
:10012000B20B9028B10B8F2808003230B100B2001A
:10013000B20B9828B10B9728080082070C340134C1
:0C014000043405340C340D340E340E343D
:02400E00F33F7E
:00000001FF
